:1000000074289400F8398C008C0C8C0C0C0C840730
:100010001320940000056F281408031C0301000638
:10002000140580066F2800308A00140807398207FB
:100030000134023404340834103420344034803421
:100040008F018E00FF308E07031C8F07031C6F2863
:1000500003308D00DF302E2022288D01E83E8C00F9
:100060008D09FC30031C37288C07031834288C07B3
:1000700064008D0F34280C183D288C1C412800008A
:100080004128080003108C0D8D0DFF3E03184228F7
:100090000C086F288D018F018E00013054288D01CE
:1000A0008F018E000430542894000F080D02031DA8
:1000B0005B280E080C0204300318013003190230CB
:1000C0001405031DFF306F280038031DFF300405A1
:1000D000031DFF306F280404031DFF306F288313B6
:1000E000031383126400080003308F00E8302120DE
:1000F0008316860185018312B201AC01AB019F28F2
:100100003108123C031DFF30FF3AA6003108593C6C
:10011000031DFF30FF3AA8002608840028086B2042
:10012000A800A90064002808290403199828B2012E
:1001300064003108143C031D9E28AC01AE01B101DE
:10014000831685140514831264000518A828A428B2
:100150006400051CAC28A828AD0164000A302D02FB
:100160000318C12864000518B628B228243084007A
:100170002D08003E01200310851803140C20AD0F3C
:10018000AD280730AD000310B10D243084002D08D8
:10019000003E01200030031D0130A600A701260803
:1001A000B1070130AD020318C3288316051083126E
:1001B000051064002E08023C031DDF28802864001F
:1001C0003108F03C031DE7280230AE009F283108BB
:1001D000123C031DFF30FF3AA6003108593C031DB5
:1001E000FF30FF3AA8002608840028086B20A800EA
:1001F000A900640028082904031901298030B200ED
:100200009F2864003108583C031D082920229F289C
:1002100064003108E03C031D0E299F28640031086A
:10022000143C031D16290230AC009F2864003108DD
:100230005A3C031D1E290D30AA00152A3208B107A9
:10024000FF30AF00FF308E008E0A0E085F3C031CAB
:10025000942930213102031D24290E08AF0094296E
:1002600001308A000E088207293496349E345D34AA
:10027000A534AE34BD345234C634C534BE34D5345E
:1002800041344E3449344A34453416341E3426340D
:1002900025342E3436343D343E344634CC344C345C
:1002A000C1345534C934CA34D2349C34B234A13444
:1002B000A334A434AB34B434B334C334BB34C23405
:1002C000CB34BA34B134C434CD349534AD349B34EA
:1002D000AC34BC34AA349D34A234B5349A3454348A
:1002E00061345B34B634CE34A6341C343234213419
:1002F000233424342B343434333443343B344234C5
:100300004B343A34313444344D3415342D341B34A9
:100310002C343C342A341D34223435341A34D43449
:10032000E134DB34DD34663464002F08FF3C031D08
:100330009A29CA2964002C08023C031DA3294030D5
:100340002F02AA00152A64002B08003C031DA929CE
:10035000122A2F088C0040304A20A6002F088C005B
:100360005B304F20A8002608840028086420A800DD
:10037000A9006400280829040319C1292F08AA002C
:10038000152A64002F081B3C031DC9293A30AA0016
:10039000152A122AFF308E008E0A0E080F3C031C0D
:1003A000EC29D8213102031DCC290E08AF00EC291D
:1003B00001308A000E0882077034693472347A344E
:1003C0006B34733474346C3475347D347C347B34E6
:1003D000793471340D34763464002F08FF3C031DEA
:1003E000F2299F282F080F3C031C112AF921AA008B
:0A03F000112A02308A002F08002AAB
:100400008207303431343234333434343534363492
:100410003734383439342A342D342B342E340934DB
:100420001B34152A20302F07AA00861702302020FF
:100430002A0886000230202086179F2863001E2A83
:1004400064002B08003C031D282A0430AB00292A35
:04045000AB010800F4
:02400E00FD3F74
:00000001FF
